:100000000C942A001895000018950000189500001F
:10001000189500001895000018950000189500002C
:10002000189500000C944A0E189500000C946B155E
:10003000189500001895000018950000189500000C
:1000400018950000189500001895000018950000FC
:10005000189500008FE181BD87E181BD8FE58DBFDF
:10006000C0E4E8E34E2E84E08EBFD4E0F4E05F2EDF
:10007000EEEFF3E0A0E6B0E088278D933197E9F743
:100080008FE289B988E18AB90E94FE136624579AE3
:100090008FE181BD87E181BD81B5886181BD877FA9
:1000A00081BDD69AA098A89A81E88FBD81E08EBDC7
:1000B0008D9A8F9A86E785BD85E083BFE1E1F0E008
:1000C000A7E9B1E091E00E944416E1E0F0E0A8E980
:1000D000B1E091E00E944416E2E0F0E0A9E9B1E06D
:1000E00091E00E944416E3E0F0E0AAE9B1E091E07B
:1000F0000E94441600EA80E2ADE9B1E00E9482135A
:10010000E4E0F0E0AFE3B2E091E00E944416EFE3F8
:10011000F2E0FA93EA935A924A9281E0A42DB52D27
:100120008C9381E00E946F130E940006249681E068
:100130000E946B13AFE3B2E08C9199279BBD8ABDFF
:10014000E5E0F0E0A0E4B2E091E00E944416A0E413
:10015000B2E08C9183BD80914002809341028091F6
:10016000400280934002E6E0F0E0A2E4B2E091E0D9
:100170000E944416E2E4F2E0FA93EA935A924A9219
:1001800080E0A42DB52D8C9381E00E946F130E9416
:100190000006249681E00E946B13E7E0F0E0A3E400
:1001A000B2E091E00E944416E8E0F0E0A4E4B2E09E
:1001B00091E00E94441604E110E020E030E0A4E465
:1001C000B2E04C915527662777270E945B14A5E47F
:1001D000B2E00D931D932D933D93EAE0F0E0A2E78A
:1001E000B2E091E00E944416E0E1F0E0AFE8B1E057
:1001F00091E00E9444168FE289B980B5807F80BD6E
:1002000000918F01013011F00C940E018FE789B934
:1002100080B5807F816080BD0C943801023011F080
:100220000C9419018FEB89B980B5807F80BD0C9447
:100230003801033011F00C9424018FE589B980B5A1
:10024000807F80BD0C943801053011F00C942F0193
:1002500087E189B980B5807F80BD0C943801063074
:1002600011F00C9438018FE089B980B5807F80BD92
:10027000A3E7B2E00E94171580E080937702EBE0DD
:10028000F0E0A8E7B2E091E00E944416ECE0F0E074
:10029000A9E7B2E091E00E944416A8E7B2E00C9111
:1002A0001127222733274CE350E060E070E00E94E2
:1002B0005B14AAE7B2E00D931D932D933D93AAE73B
:1002C000B2E00D911D912D913C91A9E7B2E04C91C6
:1002D0005527662777270E949D15AAE7B2E00D9360
:1002E0001D932D933D93AAE7B2E00D911D912D91A1
:1002F0003C914CE350E060E070E00E945B14AAE7A0
:10030000B2E00D931D932D933D93EDE0F0E0AEE749
:10031000B2E091E00E944416EEE0F0E0ABE9B2E01A
:1003200091E00E944416ABE9B2E08C9182BF7894D0
:1003300089B7816089BF89B7846089BF89B78064C4
:1003400089BF85E083BF81E08EBD86E785BD0E94C1
:10035000FE135A924A9282E0A42DB52D8C9381E02F
:100360000E946F130E949F0F229681E00E946B13E0
:1003700081E080939B0181E080939C010E94110A9F
:10038000E2E6F0E0AFE8B1E091E00E94441686E7D3
:10039000482F00918F01041711F40C94EF01ADE97F
:1003A000B1E0EEEDFCE20E948813ADE9B1E00E94FD
:1003B000D713ADE9B1E00E94D713ADE9B1E00E94D7
:1003C000D713ADE9B1E00E94D713ADE9B1E00E94C7
:1003D000D713E1E0F0E00E94F8130C94E9010E94C9
:1003E000A713ACE9B2E08C93AEE7B2E00C9102FB4C
:1003F00016F00C94FD010E943C0B00919C02003011
:1004000011F00C941902A5E4B2E04D915D916D914B
:100410007C91AFE8B2E00D911D912D913C910E942D
:10042000A7151CF011F00C9417020C9419020E94ED
:100430003C0B00919C02003011F00C942202000051
:100440000C94540200919C02013081E008F480E099
:100450008F9300919C020F3181E010F009F080E051
:100460009F918923882311F40C943A020E9456022A
:100470000C94540200919C02003881E008F480E062
:100480008F9300919C02083881E010F009F080E021
:100490009F918923882311F40C9452020E94E60E46
:1004A0000C9454020E94C1070C94EF0100919C022D
:1004B0000D3111F40C946002AFE8B2E00E94171500
:1004C00000919C02013011F00C946A020E946303B7
:1004D0000C946203023011F00C9473028AE00E94C3
:1004E0003B140C946203033011F00C947C028EE0F8
:1004F0000E943B140C946203043011F00C948402AB
:100500000E946C030C946203053011F00C948C0271
:100510000E947B030C946203063011F00C94940249
:100520000E948A030C946203073011F00C949C0221
:100530000E9499030C946203083011F00C94A402F9
:100540000E94A8030C946203093011F00C94AC02D1
:100550000E9456040C9462030A3011F00C94B40209
:100560000E945B040C9462030B3011F00C94BC02EB
:100570000E9431050C9462030C3011F00C94C402FB
:100580000E9422050C9462030D3011F00C94CC02F1
:100590000E9457050C9462030E3011F00C94D402A3
:1005A0000E945D050C9462030F3011F00C94DC0284
:1005B0000E949C050C946203013111F00C94E4023A
:1005C0000E9427060C946203023111F00C94EC0295
:1005D0000E944C060C946203033111F00C94F80253
:1005E0006894A2E7B2E08C9180F98C930C9462033A
:1005F000043111F00C940403E894A2E7B2E08C916A
:1006000080F98C930C946203053111F00C940C0367
:100610000E9477070C946203063111F00C941403C6
:100620000E947C070C946203073111F00C942003A4
:100630006894A2E7B2E08C9181F98C930C946203E8
:10064000083111F00C942C03E894A2E7B2E08C91ED
:1006500081F98C930C946203093111F00C943403EA
:100660000E9483070C9462030A3111F00C943C033E
:100670000E94BA090C9462030B3111F00C944403EC
:100680000E94FB0E0C9462030C3111F00C944C038D
:100690000E94790F0C9462030D3111F00C945403F5
:1006A0000E94C00F0C9462030E3111F00C945C0395
:1006B0000E94800F0C9462030F3111F00C946203BE
:1006C0000E94110A089581E080939B0181E080934C
:1006D0009C010E9427090895E894A2E7B2E08C915A
:1006E00082F98C93E894A2E7B2E08C9183F98C9321
:1006F0000E94270908956894A2E7B2E08C9182F9DC
:100700008C93E894A2E7B2E08C9183F98C930E94D9
:1007100027090895E894A2E7B2E08C9182F98C93BE
:100720006894A2E7B2E08C9183F98C930E94270928
:1007300008956894A2E7B2E08C9182F98C93689452
:10074000A2E7B2E08C9183F98C930E942709089567
:1007500000919C0141E0041BAEE3B2E00C930091D8
:100760003E0240919801049FAEE3B2E00C920091EA
:100770003E0240919B01040FAEE3B2E00C93AEE366
:10078000B2E08C9181508C9300913E02003011F0C8
:100790000C94F70380919A0180939C0180919801B9
:1007A00080939B0100919C0141E0041BAEE3B2E009
:1007B0000C9300913E0240919801049FAEE3B2E099
:1007C0000C9200913E0240919B01040FAEE3B2E017
:1007D0000C9331E0AEE3B2E08C918A95ADE9B1E0E3
:1007E000A80F8827B81F80E28D930C9453040091C2
:1007F0009B01013011F00C942B048091980180939F
:100800009B01ACE9B1E08C9181508C9300919C01EB
:1008100041E0041BAEE3B2E00C9300913E02409134
:100820009801049FAEE3B2E00C9200913E02409129
:100830009B01040FAEE3B2E00C9331E0AEE3B2E013
:100840008C918A95ADE9B1E0A80F8827B81F80E2A6
:100850008D930C945304ABE9B1E08C9181508C934F
:1008600000919C0141E0041BAEE3B2E00C930091C7
:100870003E0240919801049FAEE3B2E00C920091D9
:100880003E0240919B01040FAEE3B2E00C9331E0D5
:10089000AEE3B2E08C918A95ADE9B1E0A80F88276C
:1008A000B81F80E28D930E94270908950E945F136C
:1008B0000E94110A0895ACE9B1E08C918F5F8C938E
:1008C00080E08093920140919A0100919C0104176D
:1008D00018F011F00C946E040C948204A2E7B2E0BC
:1008E0000C9100FB16F00C947F04ACE9B1E08C9104
:1008F00081508C9381E0809392010C94820481E07A
:1009000080939C0100919B0140919901040FAFE8F5
:10091000B1E00C93ACE9B1E02C91AFE8B1E01C91EF
:100920000E94EB1340919A0100919C01041711F071
:100930000C941F05A2E7B2E00C9100FB16F00C949A
:100940001F0500919201013011F00C941F0581E008
:100950008093910140919C0100919101041718F03E
:1009600011F00C94F6040091910140919801049FBC
:10097000A2E9B1E00C92A2E9B1E08C918F5F8C9377
:1009800080919201EDE9F1E0009198010A93A5E6CA
:10099000B1E00E941B160091910140919801049FC3
:1009A000A2E9B1E00C920091920140919801041BE0
:1009B000A2E9B1E00C93A2E9B1E08C918F5F8C9336
:1009C000A8E9B1E03C91E5E6F1E0E8949927A2E9D5
:1009D000B1E08C91ADE9B1E00E948E13A1E9B1E0E4
:1009E0008C918F5F8C9311F00C94AA0400919C0160
:1009F00041E0041BA2E9B1E00C9300919201409107
:100A00009801049FA2E9B1E00C92A2E9B1E08C91B7
:100A10008F5F8C93A8E9B1E03C910091980180E24E
:100A2000A8E2B4E00E948213E8E2F4E0E894992797
:100A3000A2E9B1E08C91ADE9B1E00E948E130E9471
:100A40002709089581E080939B0181E080939C01B8
:100A500000EA80E2ADE9B1E00E9482130E9427091A
:100A6000089500919C0141E0041BAEE3B2E00C93B9
:100A700000913E0240919801049FAEE3B2E00C92D7
:100A800000913E0240919B01040FAEE3B2E00C9353
:100A900031E0AEE3B2E08C918A95ADE9B1E0A80F08
:100AA0008827B81F80E28D930E942709089581E06E
:100AB00080939B010E94270908950E945F13009173
:100AC0008F01043618F011F00C9468050C946B0536
:100AD00084E680938F01E5E0F0E0AFE8B1E091E0DB
:100AE0007BE70E94331600919701003011F00C94BF
:100AF000800504E640918F01041BAFE8B1E00C9340
:100B0000AFE8B1E00C9142E0049F0C9200918F019C
:100B10000A3F11F00C948F058FEF80938F01AFE89F
:100B2000B1E08C9183BD80918F01809341028091CF
:100B30008F01809340020895E2E7F0E0AFE8B1E072
:100B400091E00E94441682E6482F00918F0104171D
:100B500011F40C94CB05ADE9B1E0EEEDFCE20E949E
:100B60008813ADE9B1E00E94D713ADE9B1E00E946E
:100B7000D713ADE9B1E00E94D713ADE9B1E00E940F
:100B8000D713ADE9B1E00E94D713E1E0F0E00E9495
:100B9000F8130C94C505EFE3F2E0FA93EA930E9490
:100BA0006513229600913F02043618F011F00C9460
:100BB000DB050C94DE0584E680933F02E4E0F0E080
:100BC000AFE3B2E091E07BE70E943316EFE3F2E09F
:100BD000FA93EA935A924A9281E0A42DB52D8C9310
:100BE00081E00E946F130E940006249681E00E941B
:100BF0006B13AFE3B2E08C9199279BBD8ABD08953A
:100C0000A881B9810C91013011F00C941806AA81C9
:100C1000BB810C9142E0049F0C92AA81BB810C9194
:100C20000A3F11F00C9418068FEFAA81BB818C93B8
:100C300000919701003011F00C9426060FEFAA8165
:100C4000BB814C91041BAA81BB810C9308950E9427
:100C50005F134091980100918F01041710F00C94DC
:100C6000380600918F0141E0040FABE9B1E00C932D
:100C70000E945F1340919A0100918F01041710F0B8
:100C80000C94490600918F0141E0040FACE9B1E0FA
:100C90000C930E9427090895AFE8B2E00E9417154F
:100CA0000E945F1380918F01809393010E945F13D4
:100CB00080918F01809392010E945F1380918F0138
:100CC000809394010E945F1300918F0140919401E1
:100CD000041BA5E9B1E00C930E945F1380918F0182
:100CE000809396010E945F1380918F0180938E0103
:100CF000A3E9B1E08C9183708C9394E0A3E9B1E017
:100D00000E9401156894A3E9B1E08C9186F98C9357
:100D10005A924A9280919301A42DB52D8C9381E033
:100D20000E946F130E949F0F229681E00E946B1316
:100D3000E894A3E9B1E08C9186F98C9393E0A3E960
:100D4000B1E00E9409158FE180938F010E94450751
:100D50000091960145E00E944B16A9E8B2E08C9301
:100D600080E08093880200918902003018F011F031
:100D70000C94BC060C94CB06809189028A958093D2
:100D8000890280EF80938802A9E8B2E09C91A8E8EC
:100D9000B2E00E9409158091880280938F010E9421
:100DA00045070091960145E00E944B16A0E9B1E08D
:100DB0000C9300918E0140919801049FA6E9B1E047
:100DC0000C920091960140919401040FA6E9B1E0C4
:100DD0000C93A6E9B1E08C918F5F8C9380E08093B7
:100DE0008F014091950100918F01041718F011F0C7
:100DF0000C94420780E28093910140919001009110
:100E00008F01041710F00C940907809193018093CF
:100E100091014091900100918F01041711F00C9401
:100E200018070091930141E0040FA1E9B1E00C9390
:100E300000919101003011F00C94210788E080931B
:100E4000910131E0A1E9B1E08C91A8E2B4E08D9389
:100E500088278C93E8E2F4E0E8949927A6E9B1E0CA
:100E60008C91ADE9B1E00E948E13A6E9B1E08C91BE
:100E70008F5F8C93AFE8B1E08C918F5F8C9311F012
:100E80000C94F1060E942709089587E08093910150
:100E90004091910100E0041718F011F00C947607CE
:100EA00080E080939001A1E9B1E08C91A2E9B1E0EA
:100EB0000E9427150E941D150C900822689409F4C1
:100EC000E89416F00C94680780918F01809390014C
:100ED000A0E9B1E08C910E942B14809191018A9538
:100EE000809391018F3F11F00C94480708950E9460
:100EF0005F130E945F1308950E945F130E945F13A7
:100F00000E945F1308950E945F13AFE8B1E08C91D7
:100F100087708C9393E0AFE8B1E00E94011568946C
:100F2000AFE8B1E08C9186F98C935A924A92809105
:100F30008F01A42DB52D8C9381E00E946F130E9428
:100F40009F0F229681E00E946B130E94B6070E94B9
:100F5000B6070E94B6070E94B6070E94B6070E9415
:100F6000B6070E94B6070E94B60708950E94B11303
:100F7000AFE8B1E08C93AFE8B1E08C910E942B1404
:100F80000895AFE8B2E00E94171580E080939001C9
:100F900080E080939201A2E7B2E00C9101FB16F48D
:100FA0000C940D084091980100919B01041711F0D9
:100FB0000C940A0881E08093900100919C0141E02B
:100FC000041BAEE3B2E00C9300913E024091980105
:100FD000049FAEE3B2E00C9200913E0240919B016F
:100FE000040FAEE3B2E00C9331E0ACE9B2E08C91D7
:100FF000A8E2B4E08D9388278C93E8E2F4E0E894CB
:101000009927AEE3B2E08C91ADE9B1E00E948E1376
:101010000C940D0880E08093900180E08093920111
:1010200000919001003011F00C94880800919C010F
:1010300041E0041BAEE3B2E00C9300913E0240910C
:101040009801049FAEE3B2E00C9200913E02409101
:101050009B01040FAEE3B2E00C9331E0ACE9B2E0E7
:101060008C91A8E2B4E08D9388278C93E8E2F4E0B9
:10107000E8949927AEE3B2E08C91ADE9B1E00E942B
:101080008E13ABE9B1E08C918F5F8C934091980106
:1010900000919B01041718F011F00C9451080C9466
:1010A000780881E080939B01ACE9B1E08C918F5F7F
:1010B0008C9340919A0100919C01041718F011F053
:1010C0000C9464080C947808A2E7B2E00C9100FB41
:1010D00016F00C947508ACE9B1E08C9181508C93BA
:1010E00081E0809392010C94780881E080939C01C8
:1010F00000919B0140919901040FAFE8B1E00C937E
:10110000ACE9B1E02C91AFE8B1E01C910E94EB1387
:1011100040919A0100919C01041711F00C9421094F
:1011200000919001003011F00C94210900919B0175
:10113000013011F00C942109A2E7B2E00C9100FB00
:1011400016F00C94210900919201013011F00C94D9
:10115000210981E08093910140919C0100919101CE
:10116000041718F011F00C94F808009191014091C7
:101170009801049FA2E9B1E00C92A2E9B1E08C9140
:101180008F5F8C9380919201EDE9F1E000919801DD
:101190000A93A5E6B1E00E941B16009191014091CF
:1011A0009801049FA2E9B1E00C9200919201409154
:1011B0009801041BA2E9B1E00C93A2E9B1E08C9183
:1011C0008F5F8C93A8E9B1E03C91E5E6F1E0E8940B
:1011D0009927A2E9B1E08C91ADE9B1E00E948E13AC
:1011E000A1E9B1E08C918F5F8C9311F00C94AC0865
:1011F00000919C0141E0041BA2E9B1E00C93009135
:10120000920140919801049FA2E9B1E00C92A2E9F9
:10121000B1E08C918F5F8C93A8E9B1E03C91009193
:10122000980180E2A8E2B4E00E948213E8E2F4E0D0
:10123000E8949927A2E9B1E08C91ADE9B1E00E9470
:101240008E1380E080939C020E942709089581E01C
:1012500080938F0140919A0100918F01041718F03B
:1012600011F00C946D090091990141E0040FA0E97F
:10127000B1E00C93AFE8B1E02C91A0E9B1E01C9192
:101280000E94EB1300918F0141E0041BA0E9B1E043
:101290000C930091900140919801049FA0E9B1E066
:1012A0000C92A0E9B1E08C918F5F8C9380919001BA
:1012B000EDE9F1E0009198010A93A5E6B1E00E9402
:1012C0001B16A5E6B1E00E94D713AFE8B1E08C9100
:1012D0008F5F8C9311F00C942A09A2E7B2E00C9175
:1012E00002FB16F40C948B098EE00E943B14A2E7DB
:1012F000B2E00C9103FB16F40C9481098CE00E947F
:101300003B14A2E7B2E00C9103FB16F00C948B099E
:101310008EE00E943B14A2E7B2E00C9102FB16F0B3
:101320000C94A9098FE00E943B14A2E7B2E00C9153
:1013300003FB16F40C949F098DE00E943B14A2E776
:10134000B2E00C9103FB16F00C94A9098FE00E9407
:101350003B1400919B0140919901040FAFE8B1E06B
:101360000C93ACE9B1E02C91AFE8B1E01C910E9484
:10137000EB1308950E945F1300918F010A3111F061
:101380000C94100AA9E9B1E08C918F5F8C930E94B4
:10139000E4138FE7A9E9B1E01C910E94F513EAEF8D
:1013A000FCE20E94DD1381E880939001009190019E
:1013B000003918F011F00C94FF09A0E9B1E0EC91AC
:1013C000FF27AFE8B1E091E00E9444160091900140
:1013D00040E8041BA1E9B1E00C93A1E9B1E0EC9174
:1013E000FF27AFE8B1E091E07BE70E943316A0E968
:1013F000B1E08C918F5F8C9311F00C94D6098FEB38
:10140000A9E9B1E01C910E94F513E8E0FDE20E9419
:10141000DD1381B5886081BDEAE0F0E00E94F81339
:101420000895AFE3B2E08C9199279BBD8ABDA0E4FB
:10143000B2E08C9183BD0E94E413009198014AE0D0
:10144000041BAFE8B1E00C93AFE8B1E00C9142E0CF
:101450000E944B160C9300918F0140919901040F4B
:10146000AFE8B1E00C938FE7AFE8B1E01C910E94C8
:10147000F513E6E1FDE20E94DD138FEBAFE8B1E08A
:101480001C910E94F513E4E2FDE20E94DD138CE062
:101490000E943B1400919A01023018F011F00C9454
:1014A000530A0C94580A82E0809390010C945F0ACE
:1014B00081E080939001E5E0F0E00E94F813009154
:1014C00098014DE0041BAFE8B1E00C93AFE8B1E048
:1014D0000C9142E00E944B160C9300918F014091B9
:1014E0009901040FAFE8B1E00C93A0E9B1E02C91B1
:1014F000AFE8B1E01C910E94EB13E2E3FDE20E9431
:10150000DD13E0E1F0E0A2E9B1E091E00E944416D1
:1015100000919201013011F00C94940AE0E4FDE294
:101520000E94DD130C94C40A023011F00C949E0A40
:10153000E4E4FDE20E94DD130C94C40A033011F0D0
:101540000C94A80AE8E4FDE20E94DD130C94C40A9E
:10155000043011F00C94B20AECE4FDE20E94DD13B9
:101560000C94C40A053011F00C94BC0AE2E5FDE2CB
:101570000E94DD130C94C40A063011F00C94C40AC6
:10158000E8E5FDE20E94DD13AFE8B1E08C918F5FEA
:101590008C93A0E9B1E08C918F5F8C93A0E9B1E0CE
:1015A0002C91AFE8B1E01C910E94EB13A5E6B1E0ED
:1015B000E8E9F1E00E94C915E5E6F1E0A8E2B4E04F
:1015C0000E941616E8E2F4E0A5E6B1E01127222712
:1015D00002E033270E942D15EEE5FDE20E94DD13A7
:1015E000A5E6B1E00E94D713E2E6FDE20E94DD131A
:1015F000A5E6B1E0EAE9F1E00E94C915E5E6F1E00F
:10160000A8E2B4E00E941616E8E2F4E0A5E6B1E034
:101610001127222702E033270E942D15A5E6B1E00D
:101620000E94D713E6E6FDE20E94DD13A5E6B1E0D5
:10163000E9E9F1E00E94C915E5E6F1E0A8E2B4E0CD
:101640000E941616E8E2F4E0A5E6B1E01127222791
:1016500002E033270E942D15A5E6B1E00E94D713C2
:101660008CE00E943B14E5E0F0E00E94F8130E9439
:10167000E4130E9427090895A2E4B2E08C9199270F
:101680009BBD8ABDA3E4B2E08C9183BDE8EAF6E19C
:1016900088E40E943B1458E0C895802D0E942B14CA
:1016A00031965A95C9F704C00101010101010101F8
:1016B000ECECF6E180E50E943B1458E0C895802DE3
:1016C0000E942B1431965A95C9F704C01F010101DD
:1016D0000101011FE0EFF6E188E50E943B1458E0AC
:1016E000C895802D0E942B1431965A95C9F704C0D5
:1016F0001F1010101010101FE4E1F7E180E60E94A7
:101700003B1458E0C895802D0E942B1431965A95B1
:10171000C9F704C0111111111111111FE8E3F7E10C
:1017200088E60E943B1458E0C895802D0E942B1437
:1017300031965A95C9F704C01F1111111111111FCB
:10174000ECE5F7E180E70E943B1458E0C895802D56
:101750000E942B1431965A95C9F704C01F0101014C
:1017600001010101E0E8F7E188E70E943B1458E03D
:10177000C895802D0E942B1431965A95C9F704C044
:101780001F11111111111111E4EAF7E180E40E9417
:101790003B1458E0C895802D0E942B1431965A9521
:1017A000C9F704C02020040E0E0E0A110E94E41393
:1017B0008CE00E943B14AEE7B2E00C9101FB16F006
:1017C0000C94920C0091980144E0041BA8E8B2E04C
:1017D0000C93AEE7B2E00C9104FB16F00C94F50B01
:1017E000A8E8B2E08C9184508C93A8E8B2E00C9108
:1017F00042E00E944B160C9300918802409199019F
:10180000040FA8E8B2E00C93A3E7B2E00D911D919C
:101810002D913C9140E15EE060E070E00E94601438
:10182000AFE7B2E04D935D936D937D93A3E7B2E094
:101830000D911D912D913C9140E15EE060E070E0E2
:101840000E946014A3E8B2E00D931D932D933D9385
:10185000A3E8B2E00D911D912D913C914CE350E035
:1018600060E070E00E946014A3E8B2E04D935D93E5
:101870006D937D9300917F024AE00E944B16A7E88A
:10188000B2E00C9380E0809389020E94C50C009125
:101890007F024AE00E944B16A7E8B2E08C930E94B8
:1018A000B30C0E94C50C8BE08093870200917702F5
:1018B000003011F00C945F0C8AE0809387020E9444
:1018C000B30C0E94C50C009183024AE00E944B16A3
:1018D000A7E8B2E00C930E94B30C0E94C50C0091E3
:1018E00083024AE00E944B16A7E8B2E08C930E9464
:1018F000B30C0E94C50C8BE080938702AEE7B2E088
:101900000C9100FB16F00C94880C8CE080938702FD
:101910000E94B30C0E94C50CE894AEE7B2E08C9133
:1019200081F98C93AEE7B2E00C9102FB16F00C94B7
:101930009B0C0E94950D0E949D13082F013011F001
:101940000C94DB0BAFE3B2E08C9199279BBD8ABD71
:101950008091410280934002A0E4B2E08C9183BD6B
:101960000E9427090895A9E8B2E08C918F5F8C93BB
:10197000AEE7B2E00C9104FB16F00C94C40CA9E89D
:10198000B2E08C918F5F8C93089581E080938E02FA
:1019900000919A01043011F00C94D10C82E08093F4
:1019A0008E020091890240918802040FADE8B2E0F6
:1019B0000C93AEE8B2E02C91ADE8B2E01C910E942D
:1019C000EB1300918702013011F00C94ED0C81E0D3
:1019D00080938B0281E080938C0200918702023019
:1019E00011F00C94F90C82E080938B0283E08093D9
:1019F0008C0200918702033011F00C94050D82E0F7
:101A000080938B0282E080938C02009187020430E5
:101A100011F00C94110D84E080938B0281E080938F
:101A20008C0200918702053011F00C941D0D83E0AB
:101A300080938B0282E080938C02009187020630B3
:101A400011F00C94290D83E080938B0285E0809344
:101A50008C0200918702073011F00C94350D86E05E
:101A600080938B0281E080938C0200918702083082
:101A700011F00C94410D85E080938B0285E08093FA
:101A80008C0200918702093011F00C944D0D85E015
:101A900080938B0282E080938C0200918702003059
:101AA00011F00C94590D87E080938B0284E08093B1
:101AB0008C02009187020A3011F00C94650D81EAC6
:101AC00080938B028FED80938C02009187020B3004
:101AD00011F00C94710D80E280938B0280E2809370
:101AE0008C02009187020C3011F00C947D0D80E285
:101AF00080938B0280E080938C02ABE8B2E08C9103
:101B00000E942B14AEE8B2E08C918F5F8C93AEE80C
:101B1000B2E02C91ADE8B2E01C910E94EB13ACE86E
:101B2000B2E08C910E942B14089587E086B980EC76
:101B300087B9379AAEE8B2E02C91ADE8B2E01C91DB
:101B40000E94EB138DE00E943B1481E080938A0297
:101B500000918A02083C18F011F00C943F0E00919D
:101B60008A0248E00E944B16A7E8B2E08C930091ED
:101B70008702003011F00C94240E81E080938902DA
:101B800000918902043018F011F00C94220ED69ABC
:101B9000E4E6F0E084E690E00197DE9A0E94D21439
:101BA000DE980E94D214482F492BB1F7D69AECE266
:101BB000F1E084E690E00197DE9A0E94D214DE986C
:101BC0000E94D214482F492BB1F78AE090E00E947E
:101BD000DF14D69AE8ECF0E084E690E00197DE9A14
:101BE0000E94D214DE980E94D214482F492BB1F7DC
:101BF000D69AE8E5F2E084E690E00197DE9A0E944A
:101C0000D214DE980E94D214482F492BB1F788E2F3
:101C100090E00E94DF1487EC806C87B90E94EE147C
:101C2000082F192F043150E0150710F00C941A0EEC
:101C30000C94220EA9E8B2E08C918F5F8C9311F086
:101C40000C94C00D0C94280E82E390E00E94DF14E7
:101C500087EC806C87B90E94EE14082F192F04318D
:101C600050E0150710F00C94370E0C943F0EAAE8C4
:101C7000B2E08C918F5F8C9311F00C94A80D8CE0E6
:101C80000E943B14E894AEE7B2E08C9182F98C9309
:101C9000379808950F921F922F923F924F925F9222
:101CA0007F928F929F92AF92BF920F931F932F9329
:101CB0003F934F935F936F937F938F939F93AF93D4
:101CC000BF93CF93DF93EF93FF938FB78F938827C3
:101CD00083BFABE9B2E08C9182BFA7E7B2E08C9101
:101CE0008F5F8C93009177020C3311F00C94BA0E35
:101CF0006894AEE7B2E08C9181F98C93A3E7B2E0EF
:101D00000E947313AFE8B2E00E94731340E851E5FC
:101D100061E070E0A3E7B2E00D911D912D913C913F
:101D20000E94A71511F00C94990EA3E7B2E00E944F
:101D30001715AAE7B2E04D915D916D917C91A3E7F3
:101D4000B2E00D911D912D913C910E94A71511F0CB
:101D50000C94B70EAEE7B2E00C9100FB16F00C94B9
:101D6000B70E6894AEE7B2E08C9182F98C9380E074
:101D700080937702009177020E3111F00C94C60E19
:101D80006894AEE7B2E08C9181F98C9385E083BFD3
:101D90008F918FBFFF91EF91DF91CF91BF91AF9165
:101DA0009F918F917F916F915F914F913F912F9173
:101DB0001F910F91BF90AF909F908F907F905F90F9
:101DC0004F903F902F901F900F901895AFE8B2E082
:101DD0000E941715ACE9B2E08C9180588C93009169
:101DE0009C02003011F00C94F80E88E080939C0265
:101DF0000E94C10708950E945F130E94B113A1E6DB
:101E0000B1E08D9388278C93A1E6B1E0EAE6FDE28C
:101E10000E945B1611F00C94120FACE9B1E08C91AA
:101E200081508C93A1E6B1E0ECE6FDE20E945B16E6
:101E300011F00C94200FACE9B1E08C918F5F8C9382
:101E4000A1E6B1E0EEE6FDE20E945B1611F00C9413
:101E50002E0FABE9B1E08C918F5F8C93A1E6B1E0DE
:101E6000E0E7FDE20E945B1611F00C943C0FABE939
:101E7000B1E08C9181508C9300919B01003011F066
:101E80000C944B0FACE9B1E08C9181508C93809114
:101E9000980180939B014091980100919B01041748
:101EA00018F011F00C94560F0C945E0F81E08093A3
:101EB0009B01ACE9B1E08C918F5F8C9300919C0108
:101EC000003011F00C94680F80919A0180939C016E
:101ED00040919A0100919C01041718F011F00C94A4
:101EE000730F0C94760F81E080939C010E94C107D0
:101EF00008950E945F130E945F130E945F1308956C
:101F00000E945F1300918F01013011F00C948C0F2F
:101F10000E94B6070C949E0F0E945F135A924A9239
:101F200080918F01A42DB52D8C9381E00E946F13B9
:101F30000E949F0F229681E00E946B130895A88152
:101F4000B9810C9140EF042308BBC398C2980E944A
:101F5000BD0F94E0A881B9810E94F714A881B981CE
:101F60000C9140EF042308BBC398C2980E94BD0F98
:101F700081E090E00E94DF140895C19AC19808950D
:101F8000EEE8F1E0FA93EA930E946513229600913D
:101F90008E01013011F00C941F100E945F13AFE806
:101FA000B1E00C911127222733274CE350E060E089
:101FB00070E00E945B14A3E9B2E00D931D932D9392
:101FC0003D930E945F13A3E9B2E00D911D912D9105
:101FD0003C91AFE8B1E04C915527662777270E94E6
:101FE0009D15A3E9B2E00D931D932D933D93A3E9B5
:101FF000B2E00D911D912D913C914CE350E060E0D9
:1020000070E00E945B14A3E9B2E00D931D932D9341
:102010003D930E945F13A3E9B2E00D911D912D91B4
:102020003C91AFE8B1E04C915527662777270E9495
:102030009D15A3E7B2E00D931D932D933D93009161
:102040008E01033011F00C9471100E945F13EBE0CD
:10205000F0E0AFE8B1E091E07BE70E943316AFE833
:10206000B1E00C911127222733274CE350E060E0C8
:1020700070E00E945B14A3E9B2E00D931D932D93D1
:102080003D930E945F13ECE0F0E0AFE8B1E091E037
:102090007BE70E943316AFE8B1E00C9111272227AD
:1020A0003327A3E9B2E04D915D916D917C910E943F
:1020B0009D15A3E9B2E00D931D932D933D93A3E9E4
:1020C000B2E00D911D912D913C914CE350E060E008
:1020D00070E00E945B14AAE7B2E00D931D932D936C
:1020E0003D9300918E01053011F00C94D410E2E480
:1020F000F2E0FA93EA930E9465132296E6E0F0E09C
:10210000A2E4B2E091E07BE70E943316E2E4F2E061
:10211000FA93EA935A924A9280E0A42DB52D8C93BB
:1021200081E00E946F130E940006249681E00E94C5
:102130006B13E3E4F2E0FA93EA930E9465132296AC
:10214000E7E0F0E0A3E4B2E091E07BE70E94331621
:10215000E4E4F2E0FA93EA930E9465132296009178
:102160004402003011F00C94BA10A4E4B2E08C9157
:102170008F5F8C93E8E0F0E0A4E4B2E091E07BE7CD
:102180000E94331604E110E020E030E0A4E4B2E065
:102190004C915527662777270E945B14A5E4B2E08F
:1021A0000D931D932D933D9300918E01063011F0F8
:1021B0000C94E910EEE7F2E0FA93EA930E946513BB
:1021C0002296EDE0F0E0AEE7B2E091E07BE70E941E
:1021D000331600918E01073011F00C9414110E94F7
:1021E0005F13E1E0F0E0AFE8B1E091E07BE70E944F
:1021F00033160E945F13E2E0F0E0AFE8B1E091E057
:102200007BE70E9433160E945F13E3E0F0E0AFE843
:10221000B1E091E07BE70E94331681B5886081BD13
:10222000EAE0F0E00E94F81300918E010A3011F00C
:102230000C9452110E94E4138CE00E943B148AE03B
:1022400080938F0140918F0101E0041718F011F085
:102250000C9443118FE711E00E94F513A8E2B4E05B
:10226000EFE8F1E00E94C9150E94D51388EE93E0D3
:102270000E94DF1480918F018A9580938F018F3F98
:1022800011F00C9422118FE711E00E94F513E2E7A0
:10229000FDE20E94DD1381B5886081BDEAE0F0E0D7
:1022A0000E94F81300918E010B3011F00C94721102
:1022B0000E945F1300918F01083C18F011F00C94FC
:1022C00063110C94661188EC80938F0180918F01CB
:1022D00080939B02EEE0F0E0AFE8B1E091E07BE7B5
:1022E0000E94331600918E010C3011F00C94AB1249
:1022F000A3E9B2E00E941715A3E7B2E00D911D918A
:102300002D913C91A3E9B2E00D931D932D933C9345
:10231000A3E9B2E00D911D912D913C9140E15EE069
:1023200060E070E00E946014AFE7B2E04D935D930F
:102330006D937D93AFE7B2E00D911D912D913C918E
:1023400040E15EE060E070E00E945B14A7E9B2E06B
:102350000D931D932D933D93A3E9B2E00D911D9133
:102360002D913C91A7E9B2E04D915D916D917C91E9
:102370000E94A215A7E9B2E00D931D932D933D9302
:10238000A7E9B2E00D911D912D913C914CE350E0F5
:1023900060E070E00E946014A3E8B2E04D935D93AA
:1023A0006D937D93E0ECF3E288E40E943B1458E0E7
:1023B000C895802D0E942B1431965A95C9F704C0F8
:1023C0001B0E1517110E1120E4EEF3E280E40E94BB
:1023D0003B1458E0C895802D0E942B1431965A95D5
:1023E000C9F704C02020040E0E0E0A110E94E41347
:1023F0008CE00E943B140091980143E0041BAFE87D
:10240000B1E00C93AFE8B1E00C9142E00E944B16B2
:102410000C9300918F0140919901040FAFE8B1E056
:102420000C938FE7AFE8B1E01C910E94F51381E0B7
:102430000E942B144AE050E060E070E0AFE7B2E0A9
:102440000D911D912D913C910E94A7150CF402C095
:102450000C942E12EEE7FDE20E94DD13A8E2B4E038
:10246000EFE7F2E00E94BD150E94D513E0E8FDE21F
:102470000E94DD134AE050E060E070E0A3E8B2E0C3
:102480000D911D912D913C910E94A7150CF402C055
:102490000C944E12EEE7FDE20E94DD13A8E2B4E0D8
:1024A000E3E8F2E00E94BD150E94D5138FEBAFE880
:1024B000B1E01C910E94F513A3E9B2E00E94171548
:1024C000EBE0F0E0AFE8B1E091E00E944416ECE010
:1024D000F0E0A0E9B1E091E00E944416AEE7B2E07E
:1024E0000C9100FB16F00C947A1280E00E942B14E1
:1024F0000C947D1284E10E943B1400918F010A30FC
:1025000010F00C948712EEE7FDE20E94DD13A8E2C2
:10251000B4E0EFE8F1E00E94C9150E94D513E0E8AD
:10252000FDE20E94DD13009190010A3010F00C943E
:102530009D12EEE7FDE20E94DD13A8E2B4E0E0E9BF
:10254000F1E00E94C9150E94D513E5E0F0E00E9479
:10255000F8130E94C10700918E01013111F00C9413
:10256000C912E7E9F1E0FA93EA930E946513229613
:1025700000919701013011F40C94C11280E0809316
:102580009701E1E1F0E0A7E9B1E091E07BE70E948B
:10259000331600918E01023111F00C94FA1281E091
:1025A00080938F0100918F01003218F011F00C948C
:1025B000EF12AFE8B1E0EC91FF27A0E9B1E091E0C4
:1025C0000E944416A0E9B1E08C910E94D113AFE8BB
:1025D000B1E08C918F5F8C9311F00C94D21234E0A7
:1025E000A3E7B2E00E94CC1380E00E94D1138EE3F7
:1025F0000E94D11300918E01033111F00C945E13EF
:102600000E945F1300918F01003011F00C940B13A6
:1026100084E080938F0100918F01063018F011F053
:102620000C9414130C94171384E080938F01E0E151
:10263000F0E0AFE8B1E091E07BE70E9433168FE273
:1026400089B980B5807F80BD00918F01013011F084
:102650000C9432138FE789B980B5807F816080BD8B
:102660000C945C13023011F00C943D138FEB89B97C
:1026700080B5807F80BD0C945C13033011F00C9406
:1026800048138FE589B980B5807F80BD0C945C13B9
:10269000053011F00C94531387E189B980B5807F20
:1026A00080BD0C945C13063011F00C945C138FE029
:1026B00089B980B5807F80BD0E94110A08950E946B
:1026C000B113AFE8B1E08C9308950E94B113A881D3
:1026D000B9818C930895481A8827580A0895480E9E
:1026E0008827581E08950D911D912D913C9181E0F0
:1026F000080F8827181F281F381F3C932E931E93FE
:102700000E9308958D930A95E9F788278C93089581
:10271000C8950D9231960020D9F70895A80FB91FDA
:10272000119726F4C895802D319601C081918D9323
:10273000882311F03A95A9F7089580915F0190914F
:102740006001891711F081E00895882708959F930B
:1027500080915F019091600189179F9111F4882702
:1027600008950F929F93AF93BF9380915F019091D3
:1027700060018917D1F3A0E6B0E0A90F0024B01DD5
:102780008C9193959F3F09F4992790936001BF9195
:10279000AF919F910F9008958D9103D03A95E1F7F5
:1027A00008955D9BFECF8CB90895A8E2B4E08D91A9
:1027B000882311F050D0FBCF08950E941115802D71
:1027C00011F049D0FACF089581E055D0E4EBFBE059
:1027D0003FD080E850C08FE7213039F08FEB2230B6
:1027E00021F08FE8233009F08FEC810F0C943B141B
:1027F00088EE93E0E4D03197D9F70895882788BB15
:102800008FEF87BBECE1FEE423D080E388BBC19A65
:1028100000000000C198E4E8F3E11AD0C19A00007A
:102820000000C198E0E6F0E013D0C19A000000007B
:10283000C198E0E6F0E00CD080E288BBC19A0000CD
:102840000000C19888E217D08EE015D086E013C052
:102850003197F1F7089519D090EF982398BBC39A58
:1028600005D09FE09823929598BBC39AC19A000027
:102870000000C198089509D090EF982398BBF6DF27
:10288000829590EF982398BBF1CF9FE097BB992753
:1028900098BBC29AC19A0000000096B3C19800008C
:1028A0000000C19A00000000C19897FDEECFC298C9
:1028B0009FEF97BB089550D00AD000FC05D0089533
:1028C0004BD020D001F8F9CF52D05AD00895842FA0
:1028D000952FA62FB72F4427552766277727F1E294
:1028E000889409C020F4480F591F6A1F7B1F7695F2
:1028F0006795579547953795279517950795FA95B5
:1029000089F70895842F952FA62FB72FE894452B8C
:10291000462B472B11F468940895402F512F622FB6
:10292000732F0027112722273327F0E2440F551F6A
:10293000661F771F001F111F221F331F081B190B53
:102940002A0B3B0B416028F4080F191F2A1F3B1F5D
:102950004E7FFA9559F708950024E89477FF02C056
:1029600006D0689400F809D010F80124089512D018
:102970004F5F5F4F6F4F7F4F0895E89437FF089583
:1029800000951095209530950F5F1F4F2F4F3F4FAB
:102990006894089540955095609570950895319785
:1029A000F1F70895AE2FBF2F11974A2F4B2BE1F768
:1029B0000895689462F80895E89462F80895EF9392
:1029C000FF93EE27E82BE92B31F0E6E6FEE03197A6
:1029D000F1F70197D1F7FF91EF910895369A369963
:1029E000FECF369A3699FECF84B195B108959030D6
:1029F00039F08C91880F08F481609A95D9F78C93FF
:102A00000895903029F08C91880F9A95E9F78C936E
:102A10000895903029F08C9186959A95E9F78C93DA
:102A20000895C89531960020089582E001C084E0A1
:102A300099279D938A95E9F7089591E0882321F0DD
:102A40008894991F8A95E9F7892F90950895883081
:102A500018F011968850FBCF08952E2E3F2E9927FF
:102A600081918D3209F093958823D1F79A95E22DC3
:102A7000F32D112361F0091718F011F0101B01C09C
:102A8000191B28F021F080E28D931A95E9F78081D7
:102A90008D3219F48D93319604C0222311F08BE20C
:102AA0008D93091738F031F0091B21F080E38D93E5
:102AB0000A95E9F781918D938823E1F7332351F04B
:102AC000EA2FFB2F319633958E9182933A95E1F759
:102AD0008EE28C9308950F920F93AF93BF938F93D1
:102AE0009F938FB78F930024A0E6B0E080915F01A1
:102AF00090916001891759F49CB1A80FB01D9C9367
:102B000083958F3F09F4882780935F010DC0082FBC
:102B100003950F3F09F4002709179CB129F0A80F6E
:102B2000B01D9C9300935F018F918FBF9F918F91F8
:102B3000BF91AF910F910F901895040F151F261F8D
:102B4000371F0895041B150B260B370B0895041728
:102B50001507260737070895000F111F221F331F7F
:102B6000089500951095209530950F5F1F4F2F4FBA
:102B70003F4F0895019110810EC001911191219153
:102B800030810BC00191108117FF05C03FEF2FEF7F
:102B900004C0008111272227332737FF03C0E1DF5C
:102BA0008DE28D93CF93DF93CF92DF92EF92AA24A1
:102BB000BB24CC24DD24EE2440E2CAE0DD2755E02E
:102BC00093E38881890F87FD9F7083FD907F891B28
:102BD00089935A95A9F7C0DFAA1CBB1CCC1CDD1C2D
:102BE000EE1C4A9551F7E894EFE0FF2782910ED052
:102BF000EB30E0F71EF068948A2D0CD088278D9377
:102C0000EF90DF90CF90DF91CF910895982F82952C
:102C100001D0892F8F70805D26F0803309F40895EC
:102C200068948D93089588278D93089581918D934D
:102C30008823E1F7089509919191992351F08A959C
:102C4000D9F7319781918D930A9519F08823D1F79F
:102C50000895E9CFE199FECFEEBBFFBB3196089511
:102C600091E001C092E07B3751F47FB7F894F2DF36
:102C70008D918DBBE29AE19A9A95C9F77FBF77272C
:102C8000089591E001C092E0E5DFE09A8DB38D9365
:102C90009A95D1F70895FF93881BF9E0001FFA95E4
:102CA00011F4FF910895881F841B18F4840F8894F1
:102CB000F5CF0894F3CF689401C0E894AF93BF9325
:102CC0008D9116F0919103C00E941115902D8917D6
:102CD00018F011F48823A1F7BF91AF910895496CC2
:102CE0006C6567616C20436F7079287777772E74F5
:102CF000617669722E6875292000526573657420AB
:102D0000454550524F4D00005265626F6F74696EB9
:102D1000672E2E2E000054617649524C43442055B4
:102D2000534200007777772E74617669722E68754A
:102D3000000046773A302E363220434F4D3A00009D
:102D4000326B3400346B3800396B360031396B32FA
:102D5000000033386B34000035376B360000583ACA
:102D6000000020593A0020623A004100420043002E
:102D70004400526573746172742E2E2E0000300070
:022D80003A0017
:00000001FF
